:10000000E428040892002208840080309F0508300C
:100010009300031003189F0A1B20920C930B0A28CD
:100020000000971A1F0C1B20E22003141B201B0842
:100030008F001A0880288413971F2A28000820049C
:10004000171F20068000841700082004031C2006C8
:100050008000352800082004031C2006171B2006FA
:100060008000841720098005352817081F39FF3EB6
:100070008D001608F53E03188D0A00008D289F1389
:10008000150803199F170530940027308F00103092
:10009000552003308F00E83055208F016430552003
:1000A0008F010A30552010085C288E0011088D0041
:1000B00010088C00BE200C088C00940303199F13B9
:1000C0001508031966281402031808000C08031DFC
:1000D0009F139F1B0800303EDA28890083160814FE
:1000E00083120808DF288800831608155530890018
:1000F000AA308900881488187B280811DF288F010E
:100100008E00FF308E07031C8F07031CDF2803308F
:100110008D00DF308D2081288D01E83E8C008D0917
:10012000FC30031C96288C07031893288C07640066
:100130008D0F93280C189C288C1CA0280000A02848
:100140000800013E93000A308E008F01BE20930B01
:10015000A628100808008E000130AE2894000F0871
:100160000D02031DB5280E080C02043003180130DF
:10017000031902301405031DFF30DF28910190019F
:10018000103092000D0D900D910D0E0890020F0889
:10019000031C0F0F91020318D4280E0890070F08B4
:1001A00003180F0F910703108C0D8D0D920BC228B1
:1001B0000C08DF2884001D088A001C0882008313B5
:1001C0000313831264000800831685011330860030
:1001D000831285018601EC288501860105306D209A
:1001E000AB00861283168612643083127F2064006F
:1001F000061A22290130AA0064001F302A020318BF
:1002000008296400061A222964307F20AA0FFC28DE
:1002100064002B08013C031D10290230AB00122999
:100220000130AB00053089002B0873208616831639
:100230008612831213308F00883080208612831636
:100240008612831264002B08023C03194C2986167F
:1002500083168612831203308F00E83080208612C6
:1002600083168612831264000618332986168316B5
:10027000861206308312A2000230A000543096008D
:1002800097019A019B0131300220C8307F208612ED
:100290008316861283123329A401A5010130AA0016
:1002A000640015302A020318632986168316861205
:1002B000643083127F208612831686126430831284
:1002C0007F20AA0F5029640006186329861683161A
:1002D000861283120B308F00B8308020861283166E
:1002E000861283122C30A8000130A90028088C0047
:1002F00029088D00EA308F006030AB20031D89296A
:100300006400061C8E290A307F20A80A0319A90F51
:1003100076290B308F00B83080207229861683161C
:1003200086128312A40A0319A50A28088C0029083A
:100330008D0064308E008F01BE20A6000D08A7003E
:1003400028088C0029088D000130A120AA00280867
:100350008C0029088D000030A120AB000630A200DF
:100360000230A0005430960097019A019B0195013C
:10037000240890002508910001309C009D013F2039
:100380002C300220950126089000270891000130AA
:100390009C009D013F202E30022095012A089000EC
:1003A000910101309C009D013F2095012B08900098
:1003B000910101309C009D013F200D3002200A3048
:1003C00002200B308F00A730802086128316861201
:0803D000831272296300EA297F
:02400E00FD3F74
:02420A000200B0
:00000001FF
